ARM GAS  /tmp/ccnzHx5Q.s 			page 1


   1              		.cpu cortex-m3
   2              		.eabi_attribute 20, 1
   3              		.eabi_attribute 21, 1
   4              		.eabi_attribute 23, 3
   5              		.eabi_attribute 24, 1
   6              		.eabi_attribute 25, 1
   7              		.eabi_attribute 26, 1
   8              		.eabi_attribute 30, 1
   9              		.eabi_attribute 34, 1
  10              		.eabi_attribute 18, 4
  11              		.file	"StrBuf.c"
  12              		.text
  13              	.Ltext0:
  14              		.cfi_sections	.debug_frame
  15              		.section	.text.StrBuf_Init,"ax",%progbits
  16              		.align	1
  17              		.global	StrBuf_Init
  18              		.syntax unified
  19              		.thumb
  20              		.thumb_func
  21              		.fpu softvfp
  23              	StrBuf_Init:
  24              	.LFB0:
  25              		.file 1 "Src/StrBuf.c"
   1:Src/StrBuf.c  **** #include "StrBuf.h"
   2:Src/StrBuf.c  **** #include "utils_mod.h"
   3:Src/StrBuf.c  **** 
   4:Src/StrBuf.c  **** void StrBuf_Init(StrBuf *buf, char *array, uint16_t size)
   5:Src/StrBuf.c  **** {
  26              		.loc 1 5 0
  27              		.cfi_startproc
  28              		@ args = 0, pretend = 0, frame = 0
  29              		@ frame_needed = 0, uses_anonymous_args = 0
  30              		@ link register save eliminated.
  31              	.LVL0:
   6:Src/StrBuf.c  ****     buf->array = array;
  32              		.loc 1 6 0
  33 0000 0160     		str	r1, [r0]
   7:Src/StrBuf.c  ****     buf->size = size;
  34              		.loc 1 7 0
  35 0002 C280     		strh	r2, [r0, #6]	@ movhi
   8:Src/StrBuf.c  ****     buf->ptr = 0;
  36              		.loc 1 8 0
  37 0004 0023     		movs	r3, #0
  38 0006 8380     		strh	r3, [r0, #4]	@ movhi
   9:Src/StrBuf.c  **** }
  39              		.loc 1 9 0
  40 0008 7047     		bx	lr
  41              		.cfi_endproc
  42              	.LFE0:
  44              		.section	.text.StrBuf_Reset,"ax",%progbits
  45              		.align	1
  46              		.global	StrBuf_Reset
  47              		.syntax unified
  48              		.thumb
  49              		.thumb_func
  50              		.fpu softvfp
ARM GAS  /tmp/ccnzHx5Q.s 			page 2


  52              	StrBuf_Reset:
  53              	.LFB1:
  10:Src/StrBuf.c  **** 
  11:Src/StrBuf.c  **** void StrBuf_Reset(StrBuf *buf)
  12:Src/StrBuf.c  **** {
  54              		.loc 1 12 0
  55              		.cfi_startproc
  56              		@ args = 0, pretend = 0, frame = 0
  57              		@ frame_needed = 0, uses_anonymous_args = 0
  58              		@ link register save eliminated.
  59              	.LVL1:
  13:Src/StrBuf.c  ****     buf->ptr = 0;
  60              		.loc 1 13 0
  61 0000 0023     		movs	r3, #0
  62 0002 8380     		strh	r3, [r0, #4]	@ movhi
  14:Src/StrBuf.c  **** }
  63              		.loc 1 14 0
  64 0004 7047     		bx	lr
  65              		.cfi_endproc
  66              	.LFE1:
  68              		.section	.text.StrBuf_UsedSpace,"ax",%progbits
  69              		.align	1
  70              		.global	StrBuf_UsedSpace
  71              		.syntax unified
  72              		.thumb
  73              		.thumb_func
  74              		.fpu softvfp
  76              	StrBuf_UsedSpace:
  77              	.LFB2:
  15:Src/StrBuf.c  **** 
  16:Src/StrBuf.c  **** uint16_t StrBuf_UsedSpace(StrBuf *buf)
  17:Src/StrBuf.c  **** {
  78              		.loc 1 17 0
  79              		.cfi_startproc
  80              		@ args = 0, pretend = 0, frame = 0
  81              		@ frame_needed = 0, uses_anonymous_args = 0
  82              		@ link register save eliminated.
  83              	.LVL2:
  18:Src/StrBuf.c  ****     return buf->ptr;
  19:Src/StrBuf.c  **** }
  84              		.loc 1 19 0
  85 0000 8088     		ldrh	r0, [r0, #4]
  86              	.LVL3:
  87 0002 7047     		bx	lr
  88              		.cfi_endproc
  89              	.LFE2:
  91              		.section	.text.StrBuf_RemainingSpace,"ax",%progbits
  92              		.align	1
  93              		.global	StrBuf_RemainingSpace
  94              		.syntax unified
  95              		.thumb
  96              		.thumb_func
  97              		.fpu softvfp
  99              	StrBuf_RemainingSpace:
 100              	.LFB3:
  20:Src/StrBuf.c  **** 
  21:Src/StrBuf.c  **** uint16_t StrBuf_RemainingSpace(StrBuf *buf)
ARM GAS  /tmp/ccnzHx5Q.s 			page 3


  22:Src/StrBuf.c  **** {
 101              		.loc 1 22 0
 102              		.cfi_startproc
 103              		@ args = 0, pretend = 0, frame = 0
 104              		@ frame_needed = 0, uses_anonymous_args = 0
 105              		@ link register save eliminated.
 106              	.LVL4:
  23:Src/StrBuf.c  ****     return buf->size - buf->ptr;
 107              		.loc 1 23 0
 108 0000 C388     		ldrh	r3, [r0, #6]
 109 0002 8088     		ldrh	r0, [r0, #4]
 110              	.LVL5:
 111 0004 181A     		subs	r0, r3, r0
  24:Src/StrBuf.c  **** }
 112              		.loc 1 24 0
 113 0006 80B2     		uxth	r0, r0
 114 0008 7047     		bx	lr
 115              		.cfi_endproc
 116              	.LFE3:
 118              		.section	.text.StrBuf_Capacity,"ax",%progbits
 119              		.align	1
 120              		.global	StrBuf_Capacity
 121              		.syntax unified
 122              		.thumb
 123              		.thumb_func
 124              		.fpu softvfp
 126              	StrBuf_Capacity:
 127              	.LFB4:
  25:Src/StrBuf.c  **** 
  26:Src/StrBuf.c  **** uint16_t StrBuf_Capacity(StrBuf *buf)
  27:Src/StrBuf.c  **** {
 128              		.loc 1 27 0
 129              		.cfi_startproc
 130              		@ args = 0, pretend = 0, frame = 0
 131              		@ frame_needed = 0, uses_anonymous_args = 0
 132              		@ link register save eliminated.
 133              	.LVL6:
  28:Src/StrBuf.c  ****     return buf->size;
  29:Src/StrBuf.c  **** }
 134              		.loc 1 29 0
 135 0000 C088     		ldrh	r0, [r0, #6]
 136              	.LVL7:
 137 0002 7047     		bx	lr
 138              		.cfi_endproc
 139              	.LFE4:
 141              		.section	.text.StrBuf_Array,"ax",%progbits
 142              		.align	1
 143              		.global	StrBuf_Array
 144              		.syntax unified
 145              		.thumb
 146              		.thumb_func
 147              		.fpu softvfp
 149              	StrBuf_Array:
 150              	.LFB5:
  30:Src/StrBuf.c  **** 
  31:Src/StrBuf.c  **** char* StrBuf_Array(StrBuf *buf)
  32:Src/StrBuf.c  **** {
ARM GAS  /tmp/ccnzHx5Q.s 			page 4


 151              		.loc 1 32 0
 152              		.cfi_startproc
 153              		@ args = 0, pretend = 0, frame = 0
 154              		@ frame_needed = 0, uses_anonymous_args = 0
 155              		@ link register save eliminated.
 156              	.LVL8:
  33:Src/StrBuf.c  ****     return buf->array;
  34:Src/StrBuf.c  **** }
 157              		.loc 1 34 0
 158 0000 0068     		ldr	r0, [r0]
 159              	.LVL9:
 160 0002 7047     		bx	lr
 161              		.cfi_endproc
 162              	.LFE5:
 164              		.section	.text.StrBuf_UInt32,"ax",%progbits
 165              		.align	1
 166              		.global	StrBuf_UInt32
 167              		.syntax unified
 168              		.thumb
 169              		.thumb_func
 170              		.fpu softvfp
 172              	StrBuf_UInt32:
 173              	.LFB6:
  35:Src/StrBuf.c  **** 
  36:Src/StrBuf.c  **** void StrBuf_UInt32(StrBuf *buf, uint32_t number)
  37:Src/StrBuf.c  **** {
 174              		.loc 1 37 0
 175              		.cfi_startproc
 176              		@ args = 0, pretend = 0, frame = 0
 177              		@ frame_needed = 0, uses_anonymous_args = 0
 178              	.LVL10:
 179 0000 F8B5     		push	{r3, r4, r5, r6, r7, lr}
 180              	.LCFI0:
 181              		.cfi_def_cfa_offset 24
 182              		.cfi_offset 3, -24
 183              		.cfi_offset 4, -20
 184              		.cfi_offset 5, -16
 185              		.cfi_offset 6, -12
 186              		.cfi_offset 7, -8
 187              		.cfi_offset 14, -4
 188              	.LVL11:
  38:Src/StrBuf.c  ****     uint8_t nonzero_found = 0;
  39:Src/StrBuf.c  **** 
  40:Src/StrBuf.c  ****     if(number == 0) {
 189              		.loc 1 40 0
 190 0002 0029     		cmp	r1, #0
 191 0004 32D1     		bne	.L13
  41:Src/StrBuf.c  ****         if(buf->ptr < buf->size)
 192              		.loc 1 41 0
 193 0006 8388     		ldrh	r3, [r0, #4]
 194 0008 C288     		ldrh	r2, [r0, #6]
 195 000a 9342     		cmp	r3, r2
 196 000c 04D2     		bcs	.L7
  42:Src/StrBuf.c  ****             buf->array[(buf->ptr)++] = '0';
 197              		.loc 1 42 0
 198 000e 0268     		ldr	r2, [r0]
 199 0010 591C     		adds	r1, r3, #1
ARM GAS  /tmp/ccnzHx5Q.s 			page 5


 200              	.LVL12:
 201 0012 8180     		strh	r1, [r0, #4]	@ movhi
 202 0014 3021     		movs	r1, #48
 203 0016 D154     		strb	r1, [r2, r3]
 204              	.LVL13:
 205              	.L7:
  43:Src/StrBuf.c  ****         return;
  44:Src/StrBuf.c  ****     }
  45:Src/StrBuf.c  **** 
  46:Src/StrBuf.c  ****     for(uint16_t i = 0; i < 10 && buf->ptr < buf->size; ++i) {
  47:Src/StrBuf.c  ****         uint8_t digit = (number / cpow10(9-i)) % 10;
  48:Src/StrBuf.c  ****         if(digit) {
  49:Src/StrBuf.c  ****             nonzero_found = 1;
  50:Src/StrBuf.c  ****             buf->array[(buf->ptr)++] = '0' + digit;
  51:Src/StrBuf.c  ****         } else {
  52:Src/StrBuf.c  ****             if(nonzero_found)
  53:Src/StrBuf.c  ****                 buf->array[(buf->ptr)++] = '0' + digit;
  54:Src/StrBuf.c  ****         }
  55:Src/StrBuf.c  ****     }
  56:Src/StrBuf.c  **** }
 206              		.loc 1 56 0
 207 0018 F8BD     		pop	{r3, r4, r5, r6, r7, pc}
 208              	.LVL14:
 209              	.L10:
 210              	.LBB2:
 211              	.LBB3:
  52:Src/StrBuf.c  ****                 buf->array[(buf->ptr)++] = '0' + digit;
 212              		.loc 1 52 0
 213 001a 2FB1     		cbz	r7, .L11
  53:Src/StrBuf.c  ****         }
 214              		.loc 1 53 0
 215 001c 2968     		ldr	r1, [r5]
 216 001e AA88     		ldrh	r2, [r5, #4]
 217              	.LVL15:
 218 0020 501C     		adds	r0, r2, #1
 219              	.LVL16:
 220 0022 A880     		strh	r0, [r5, #4]	@ movhi
 221 0024 3033     		adds	r3, r3, #48
 222 0026 8B54     		strb	r3, [r1, r2]
 223              	.LVL17:
 224              	.L11:
 225              	.LBE3:
  46:Src/StrBuf.c  ****         uint8_t digit = (number / cpow10(9-i)) % 10;
 226              		.loc 1 46 0 discriminator 2
 227 0028 0134     		adds	r4, r4, #1
 228              	.LVL18:
 229 002a A4B2     		uxth	r4, r4
 230              	.LVL19:
 231              	.L8:
  46:Src/StrBuf.c  ****         uint8_t digit = (number / cpow10(9-i)) % 10;
 232              		.loc 1 46 0 is_stmt 0 discriminator 1
 233 002c 092C     		cmp	r4, #9
 234 002e F3D8     		bhi	.L7
  46:Src/StrBuf.c  ****         uint8_t digit = (number / cpow10(9-i)) % 10;
 235              		.loc 1 46 0 discriminator 3
 236 0030 AA88     		ldrh	r2, [r5, #4]
 237 0032 EB88     		ldrh	r3, [r5, #6]
ARM GAS  /tmp/ccnzHx5Q.s 			page 6


 238 0034 9A42     		cmp	r2, r3
 239 0036 EFD2     		bcs	.L7
 240              	.LBB4:
  47:Src/StrBuf.c  ****         if(digit) {
 241              		.loc 1 47 0 is_stmt 1
 242 0038 C4F10900 		rsb	r0, r4, #9
 243 003c C0B2     		uxtb	r0, r0
 244 003e FFF7FEFF 		bl	cpow10
 245              	.LVL20:
 246 0042 B6FBF0F0 		udiv	r0, r6, r0
 247 0046 0C4B     		ldr	r3, .L15
 248 0048 A3FB0023 		umull	r2, r3, r3, r0
 249 004c DB08     		lsrs	r3, r3, #3
 250 004e 03EB8303 		add	r3, r3, r3, lsl #2
 251 0052 5A00     		lsls	r2, r3, #1
 252 0054 831A     		subs	r3, r0, r2
 253              	.LVL21:
  48:Src/StrBuf.c  ****             nonzero_found = 1;
 254              		.loc 1 48 0
 255 0056 13F0FF03 		ands	r3, r3, #255
 256              	.LVL22:
 257 005a DED0     		beq	.L10
 258              	.LVL23:
  50:Src/StrBuf.c  ****         } else {
 259              		.loc 1 50 0
 260 005c 2968     		ldr	r1, [r5]
 261 005e AA88     		ldrh	r2, [r5, #4]
 262              	.LVL24:
 263 0060 501C     		adds	r0, r2, #1
 264              	.LVL25:
 265 0062 A880     		strh	r0, [r5, #4]	@ movhi
 266 0064 3033     		adds	r3, r3, #48
 267 0066 8B54     		strb	r3, [r1, r2]
  49:Src/StrBuf.c  ****             buf->array[(buf->ptr)++] = '0' + digit;
 268              		.loc 1 49 0
 269 0068 0127     		movs	r7, #1
 270 006a DDE7     		b	.L11
 271              	.LVL26:
 272              	.L13:
 273 006c 0E46     		mov	r6, r1
 274 006e 0546     		mov	r5, r0
 275              	.LBE4:
  46:Src/StrBuf.c  ****         uint8_t digit = (number / cpow10(9-i)) % 10;
 276              		.loc 1 46 0
 277 0070 0024     		movs	r4, #0
 278              	.LBE2:
  38:Src/StrBuf.c  **** 
 279              		.loc 1 38 0
 280 0072 2746     		mov	r7, r4
 281 0074 DAE7     		b	.L8
 282              	.L16:
 283 0076 00BF     		.align	2
 284              	.L15:
 285 0078 CDCCCCCC 		.word	-858993459
 286              		.cfi_endproc
 287              	.LFE6:
 289              		.section	.text.StrBuf_UInt32Bin,"ax",%progbits
ARM GAS  /tmp/ccnzHx5Q.s 			page 7


 290              		.align	1
 291              		.global	StrBuf_UInt32Bin
 292              		.syntax unified
 293              		.thumb
 294              		.thumb_func
 295              		.fpu softvfp
 297              	StrBuf_UInt32Bin:
 298              	.LFB7:
  57:Src/StrBuf.c  **** 
  58:Src/StrBuf.c  **** void StrBuf_UInt32Bin(StrBuf *buf, uint32_t number, bool zero_fill)
  59:Src/StrBuf.c  **** {
 299              		.loc 1 59 0
 300              		.cfi_startproc
 301              		@ args = 0, pretend = 0, frame = 0
 302              		@ frame_needed = 0, uses_anonymous_args = 0
 303              		@ link register save eliminated.
 304              	.LVL27:
 305 0000 F0B4     		push	{r4, r5, r6, r7}
 306              	.LCFI1:
 307              		.cfi_def_cfa_offset 16
 308              		.cfi_offset 4, -16
 309              		.cfi_offset 5, -12
 310              		.cfi_offset 6, -8
 311              		.cfi_offset 7, -4
 312              	.LVL28:
  60:Src/StrBuf.c  ****     uint8_t nonzero_found = 0;
  61:Src/StrBuf.c  **** 
  62:Src/StrBuf.c  ****     if(number == 0) {
 313              		.loc 1 62 0
 314 0002 19B1     		cbz	r1, .L27
 315 0004 0D46     		mov	r5, r1
 316              	.LBB5:
  63:Src/StrBuf.c  ****         for(uint8_t i = 0; i < (zero_fill ? 32 : 1) && buf->ptr < buf->size; ++i)
  64:Src/StrBuf.c  ****             buf->array[(buf->ptr)++] = '0';
  65:Src/StrBuf.c  ****         return;
  66:Src/StrBuf.c  ****     }
  67:Src/StrBuf.c  **** 
  68:Src/StrBuf.c  ****     for(uint16_t i = 0u; i < 32u && buf->ptr < buf->size; ++i) {
 317              		.loc 1 68 0
 318 0006 0021     		movs	r1, #0
 319              	.LVL29:
 320              	.LBE5:
  60:Src/StrBuf.c  ****     uint8_t nonzero_found = 0;
 321              		.loc 1 60 0
 322 0008 0F46     		mov	r7, r1
 323 000a 1FE0     		b	.L19
 324              	.LVL30:
 325              	.L27:
 326              	.LBB8:
  63:Src/StrBuf.c  ****         for(uint8_t i = 0; i < (zero_fill ? 32 : 1) && buf->ptr < buf->size; ++i)
 327              		.loc 1 63 0
 328 000c 0023     		movs	r3, #0
 329 000e 0DE0     		b	.L18
 330              	.LVL31:
 331              	.L28:
 332 0010 0124     		movs	r4, #1
 333              	.L20:
ARM GAS  /tmp/ccnzHx5Q.s 			page 8


  63:Src/StrBuf.c  ****         for(uint8_t i = 0; i < (zero_fill ? 32 : 1) && buf->ptr < buf->size; ++i)
 334              		.loc 1 63 0 is_stmt 0 discriminator 6
 335 0012 A142     		cmp	r1, r4
 336 0014 2EDA     		bge	.L17
  63:Src/StrBuf.c  ****         for(uint8_t i = 0; i < (zero_fill ? 32 : 1) && buf->ptr < buf->size; ++i)
 337              		.loc 1 63 0 discriminator 7
 338 0016 8188     		ldrh	r1, [r0, #4]
 339 0018 C488     		ldrh	r4, [r0, #6]
 340 001a A142     		cmp	r1, r4
 341 001c 2AD2     		bcs	.L17
  64:Src/StrBuf.c  ****         return;
 342              		.loc 1 64 0 is_stmt 1 discriminator 8
 343 001e 0468     		ldr	r4, [r0]
 344 0020 4D1C     		adds	r5, r1, #1
 345 0022 8580     		strh	r5, [r0, #4]	@ movhi
 346 0024 3025     		movs	r5, #48
 347 0026 6554     		strb	r5, [r4, r1]
  63:Src/StrBuf.c  ****         for(uint8_t i = 0; i < (zero_fill ? 32 : 1) && buf->ptr < buf->size; ++i)
 348              		.loc 1 63 0 discriminator 8
 349 0028 0133     		adds	r3, r3, #1
 350              	.LVL32:
 351 002a DBB2     		uxtb	r3, r3
 352              	.LVL33:
 353              	.L18:
  63:Src/StrBuf.c  ****         for(uint8_t i = 0; i < (zero_fill ? 32 : 1) && buf->ptr < buf->size; ++i)
 354              		.loc 1 63 0 is_stmt 0 discriminator 1
 355 002c 1946     		mov	r1, r3
 356 002e 002A     		cmp	r2, #0
 357 0030 EED0     		beq	.L28
  63:Src/StrBuf.c  ****         for(uint8_t i = 0; i < (zero_fill ? 32 : 1) && buf->ptr < buf->size; ++i)
 358              		.loc 1 63 0
 359 0032 2024     		movs	r4, #32
 360 0034 EDE7     		b	.L20
 361              	.LVL34:
 362              	.L23:
 363              	.LBE8:
 364              	.LBB9:
 365              	.LBB6:
  69:Src/StrBuf.c  ****         uint8_t digit = (number >> (31u-i)) & 1u;
  70:Src/StrBuf.c  ****         if(digit) {
  71:Src/StrBuf.c  ****             nonzero_found = 1;
  72:Src/StrBuf.c  ****             buf->array[(buf->ptr)++] = '0' + digit;
  73:Src/StrBuf.c  ****         } else {
  74:Src/StrBuf.c  ****             if(nonzero_found || zero_fill)
 366              		.loc 1 74 0 is_stmt 1
 367 0036 07B9     		cbnz	r7, .L25
 368              		.loc 1 74 0 is_stmt 0 discriminator 1
 369 0038 32B1     		cbz	r2, .L24
 370              	.L25:
  75:Src/StrBuf.c  ****                 buf->array[(buf->ptr)++] = '0' + digit;
 371              		.loc 1 75 0 is_stmt 1
 372 003a 0668     		ldr	r6, [r0]
 373 003c 04F1010C 		add	ip, r4, #1
 374 0040 A0F804C0 		strh	ip, [r0, #4]	@ movhi
 375 0044 3033     		adds	r3, r3, #48
 376 0046 3355     		strb	r3, [r6, r4]
 377              	.LVL35:
ARM GAS  /tmp/ccnzHx5Q.s 			page 9


 378              	.L24:
 379              	.LBE6:
  68:Src/StrBuf.c  ****         uint8_t digit = (number >> (31u-i)) & 1u;
 380              		.loc 1 68 0 discriminator 2
 381 0048 0131     		adds	r1, r1, #1
 382              	.LVL36:
 383 004a 89B2     		uxth	r1, r1
 384              	.LVL37:
 385              	.L19:
  68:Src/StrBuf.c  ****         uint8_t digit = (number >> (31u-i)) & 1u;
 386              		.loc 1 68 0 is_stmt 0 discriminator 1
 387 004c 1F29     		cmp	r1, #31
 388 004e 11D8     		bhi	.L17
  68:Src/StrBuf.c  ****         uint8_t digit = (number >> (31u-i)) & 1u;
 389              		.loc 1 68 0 discriminator 3
 390 0050 8488     		ldrh	r4, [r0, #4]
 391 0052 C388     		ldrh	r3, [r0, #6]
 392 0054 9C42     		cmp	r4, r3
 393 0056 0DD2     		bcs	.L17
 394              	.LBB7:
  69:Src/StrBuf.c  ****         uint8_t digit = (number >> (31u-i)) & 1u;
 395              		.loc 1 69 0 is_stmt 1
 396 0058 C1F11F03 		rsb	r3, r1, #31
 397 005c 25FA03F3 		lsr	r3, r5, r3
 398              	.LVL38:
  70:Src/StrBuf.c  ****             nonzero_found = 1;
 399              		.loc 1 70 0
 400 0060 13F00103 		ands	r3, r3, #1
 401              	.LVL39:
 402 0064 E7D0     		beq	.L23
 403              	.LVL40:
  72:Src/StrBuf.c  ****         } else {
 404              		.loc 1 72 0
 405 0066 0668     		ldr	r6, [r0]
 406 0068 671C     		adds	r7, r4, #1
 407 006a 8780     		strh	r7, [r0, #4]	@ movhi
 408 006c 3033     		adds	r3, r3, #48
 409 006e 3355     		strb	r3, [r6, r4]
  71:Src/StrBuf.c  ****             buf->array[(buf->ptr)++] = '0' + digit;
 410              		.loc 1 71 0
 411 0070 0127     		movs	r7, #1
 412 0072 E9E7     		b	.L24
 413              	.LVL41:
 414              	.L17:
 415              	.LBE7:
 416              	.LBE9:
  76:Src/StrBuf.c  ****         }
  77:Src/StrBuf.c  ****     }
  78:Src/StrBuf.c  **** }
 417              		.loc 1 78 0
 418 0074 F0BC     		pop	{r4, r5, r6, r7}
 419              	.LCFI2:
 420              		.cfi_restore 7
 421              		.cfi_restore 6
 422              		.cfi_restore 5
 423              		.cfi_restore 4
 424              		.cfi_def_cfa_offset 0
ARM GAS  /tmp/ccnzHx5Q.s 			page 10


 425 0076 7047     		bx	lr
 426              		.cfi_endproc
 427              	.LFE7:
 429              		.global	__aeabi_f2uiz
 430              		.global	__aeabi_ui2f
 431              		.global	__aeabi_fsub
 432              		.global	__aeabi_fmul
 433              		.section	.text.StrBuf_Float,"ax",%progbits
 434              		.align	1
 435              		.global	StrBuf_Float
 436              		.syntax unified
 437              		.thumb
 438              		.thumb_func
 439              		.fpu softvfp
 441              	StrBuf_Float:
 442              	.LFB8:
  79:Src/StrBuf.c  **** 
  80:Src/StrBuf.c  **** void StrBuf_Float(StrBuf *buf, float number, uint8_t precision)
  81:Src/StrBuf.c  **** {
 443              		.loc 1 81 0
 444              		.cfi_startproc
 445              		@ args = 0, pretend = 0, frame = 24
 446              		@ frame_needed = 0, uses_anonymous_args = 0
 447              	.LVL42:
 448 0000 2DE9F04F 		push	{r4, r5, r6, r7, r8, r9, r10, fp, lr}
 449              	.LCFI3:
 450              		.cfi_def_cfa_offset 36
 451              		.cfi_offset 4, -36
 452              		.cfi_offset 5, -32
 453              		.cfi_offset 6, -28
 454              		.cfi_offset 7, -24
 455              		.cfi_offset 8, -20
 456              		.cfi_offset 9, -16
 457              		.cfi_offset 10, -12
 458              		.cfi_offset 11, -8
 459              		.cfi_offset 14, -4
 460 0004 87B0     		sub	sp, sp, #28
 461              	.LCFI4:
 462              		.cfi_def_cfa_offset 64
 463 0006 0546     		mov	r5, r0
 464 0008 8946     		mov	r9, r1
 465 000a 1646     		mov	r6, r2
  82:Src/StrBuf.c  ****     StrBuf_UInt32(buf, (uint32_t)number);
 466              		.loc 1 82 0
 467 000c 0846     		mov	r0, r1
 468              	.LVL43:
 469 000e FFF7FEFF 		bl	__aeabi_f2uiz
 470              	.LVL44:
 471 0012 8046     		mov	r8, r0
 472 0014 0146     		mov	r1, r0
 473 0016 2846     		mov	r0, r5
 474 0018 FFF7FEFF 		bl	StrBuf_UInt32
 475              	.LVL45:
  83:Src/StrBuf.c  **** 
  84:Src/StrBuf.c  ****     if(buf->ptr >= buf->size)
 476              		.loc 1 84 0
 477 001c AB88     		ldrh	r3, [r5, #4]
ARM GAS  /tmp/ccnzHx5Q.s 			page 11


 478 001e EA88     		ldrh	r2, [r5, #6]
 479 0020 9342     		cmp	r3, r2
 480 0022 5FD2     		bcs	.L30
  85:Src/StrBuf.c  ****         return;
  86:Src/StrBuf.c  **** 
  87:Src/StrBuf.c  ****     buf->array[(buf->ptr)++] = '.';
 481              		.loc 1 87 0
 482 0024 2A68     		ldr	r2, [r5]
 483 0026 591C     		adds	r1, r3, #1
 484 0028 A980     		strh	r1, [r5, #4]	@ movhi
 485 002a 2E21     		movs	r1, #46
 486 002c D154     		strb	r1, [r2, r3]
  88:Src/StrBuf.c  **** 
  89:Src/StrBuf.c  ****     char frac_digits[20];
  90:Src/StrBuf.c  ****     if(precision > 20)
 487              		.loc 1 90 0
 488 002e 142E     		cmp	r6, #20
 489 0030 00D9     		bls	.L32
  91:Src/StrBuf.c  ****         precision = 20;
 490              		.loc 1 91 0
 491 0032 1426     		movs	r6, #20
 492              	.L32:
 493              	.LVL46:
 494              	.LBB10:
  92:Src/StrBuf.c  **** 
  93:Src/StrBuf.c  ****     uint8_t dig0_cnt = 0;
  94:Src/StrBuf.c  ****     uint8_t nonzero_found = 0;
  95:Src/StrBuf.c  **** 
  96:Src/StrBuf.c  ****     for(uint8_t i = 0; i < precision; ++i) {
 495              		.loc 1 96 0
 496 0034 0024     		movs	r4, #0
 497              	.LBE10:
  94:Src/StrBuf.c  **** 
 498              		.loc 1 94 0
 499 0036 A246     		mov	r10, r4
  93:Src/StrBuf.c  ****     uint8_t nonzero_found = 0;
 500              		.loc 1 93 0
 501 0038 2746     		mov	r7, r4
 502              	.LBB13:
 503              		.loc 1 96 0
 504 003a 03E0     		b	.L33
 505              	.LVL47:
 506              	.L41:
 507              	.LBB11:
  97:Src/StrBuf.c  ****         float num = (number - (uint32_t)number) * cpow10(precision-i);
  98:Src/StrBuf.c  ****         uint8_t digit = (uint32_t)num % 10;
  99:Src/StrBuf.c  ****         frac_digits[i] = '0' + digit;
 100:Src/StrBuf.c  **** 
 101:Src/StrBuf.c  ****         if(digit != 0)
 102:Src/StrBuf.c  ****             nonzero_found = 1;
 508              		.loc 1 102 0
 509 003c 4FF0010A 		mov	r10, #1
 510              	.LVL48:
 511              	.L34:
 512              	.LBE11:
  96:Src/StrBuf.c  ****         float num = (number - (uint32_t)number) * cpow10(precision-i);
 513              		.loc 1 96 0 discriminator 2
ARM GAS  /tmp/ccnzHx5Q.s 			page 12


 514 0040 0134     		adds	r4, r4, #1
 515              	.LVL49:
 516 0042 E4B2     		uxtb	r4, r4
 517              	.LVL50:
 518              	.L33:
  96:Src/StrBuf.c  ****         float num = (number - (uint32_t)number) * cpow10(precision-i);
 519              		.loc 1 96 0 is_stmt 0 discriminator 1
 520 0044 A642     		cmp	r6, r4
 521 0046 2AD9     		bls	.L44
 522              	.LBB12:
  97:Src/StrBuf.c  ****         float num = (number - (uint32_t)number) * cpow10(precision-i);
 523              		.loc 1 97 0 is_stmt 1
 524 0048 4046     		mov	r0, r8
 525 004a FFF7FEFF 		bl	__aeabi_ui2f
 526              	.LVL51:
 527 004e 0146     		mov	r1, r0
 528 0050 4846     		mov	r0, r9
 529 0052 FFF7FEFF 		bl	__aeabi_fsub
 530              	.LVL52:
 531 0056 8346     		mov	fp, r0
 532 0058 301B     		subs	r0, r6, r4
 533 005a C0B2     		uxtb	r0, r0
 534 005c FFF7FEFF 		bl	cpow10
 535              	.LVL53:
 536 0060 FFF7FEFF 		bl	__aeabi_ui2f
 537              	.LVL54:
 538 0064 0146     		mov	r1, r0
 539 0066 5846     		mov	r0, fp
 540 0068 FFF7FEFF 		bl	__aeabi_fmul
 541              	.LVL55:
  98:Src/StrBuf.c  ****         frac_digits[i] = '0' + digit;
 542              		.loc 1 98 0
 543 006c FFF7FEFF 		bl	__aeabi_f2uiz
 544              	.LVL56:
 545 0070 1E4B     		ldr	r3, .L46
 546 0072 A3FB0023 		umull	r2, r3, r3, r0
 547 0076 DB08     		lsrs	r3, r3, #3
 548 0078 03EB8303 		add	r3, r3, r3, lsl #2
 549 007c 5A00     		lsls	r2, r3, #1
 550 007e 831A     		subs	r3, r0, r2
 551 0080 DBB2     		uxtb	r3, r3
 552              	.LVL57:
  99:Src/StrBuf.c  **** 
 553              		.loc 1 99 0
 554 0082 03F13001 		add	r1, r3, #48
 555 0086 06AA     		add	r2, sp, #24
 556 0088 2244     		add	r2, r2, r4
 557 008a 02F8141C 		strb	r1, [r2, #-20]
 101:Src/StrBuf.c  ****             nonzero_found = 1;
 558              		.loc 1 101 0
 559 008e 002B     		cmp	r3, #0
 560 0090 D4D1     		bne	.L41
 103:Src/StrBuf.c  ****         if(!nonzero_found)
 561              		.loc 1 103 0
 562 0092 BAF1000F 		cmp	r10, #0
 563 0096 D3D1     		bne	.L34
 104:Src/StrBuf.c  ****             dig0_cnt++;
ARM GAS  /tmp/ccnzHx5Q.s 			page 13


 564              		.loc 1 104 0
 565 0098 0137     		adds	r7, r7, #1
 566              	.LVL58:
 567 009a FFB2     		uxtb	r7, r7
 568              	.LVL59:
 569 009c D0E7     		b	.L34
 570              	.LVL60:
 571              	.L44:
 572              	.LBE12:
 573              	.LBE13:
 105:Src/StrBuf.c  ****     }
 106:Src/StrBuf.c  **** 
 107:Src/StrBuf.c  ****     if(dig0_cnt == precision) {
 574              		.loc 1 107 0
 575 009e BE42     		cmp	r6, r7
 576 00a0 01D0     		beq	.L45
 577              	.LBB14:
 108:Src/StrBuf.c  ****         if(buf->ptr < buf->size)
 109:Src/StrBuf.c  ****             buf->array[(buf->ptr)++] = '0';
 110:Src/StrBuf.c  ****     } else {
 111:Src/StrBuf.c  ****         for(uint8_t i = 0; i < precision-dig0_cnt && buf->ptr < buf->size; ++i)
 578              		.loc 1 111 0
 579 00a2 0022     		movs	r2, #0
 580 00a4 15E0     		b	.L36
 581              	.L45:
 582              	.LBE14:
 108:Src/StrBuf.c  ****         if(buf->ptr < buf->size)
 583              		.loc 1 108 0
 584 00a6 AB88     		ldrh	r3, [r5, #4]
 585 00a8 EA88     		ldrh	r2, [r5, #6]
 586 00aa 9342     		cmp	r3, r2
 587 00ac 1AD2     		bcs	.L30
 109:Src/StrBuf.c  ****     } else {
 588              		.loc 1 109 0
 589 00ae 2A68     		ldr	r2, [r5]
 590 00b0 591C     		adds	r1, r3, #1
 591 00b2 A980     		strh	r1, [r5, #4]	@ movhi
 592 00b4 3021     		movs	r1, #48
 593 00b6 D154     		strb	r1, [r2, r3]
 594 00b8 14E0     		b	.L30
 595              	.LVL61:
 596              	.L38:
 597              	.LBB15:
 112:Src/StrBuf.c  ****             buf->array[(buf->ptr)++] = frac_digits[precision-1-i];
 598              		.loc 1 112 0 discriminator 4
 599 00ba 013B     		subs	r3, r3, #1
 600 00bc 1B1A     		subs	r3, r3, r0
 601 00be 2868     		ldr	r0, [r5]
 602 00c0 4C1C     		adds	r4, r1, #1
 603 00c2 AC80     		strh	r4, [r5, #4]	@ movhi
 604 00c4 06AC     		add	r4, sp, #24
 605 00c6 2344     		add	r3, r3, r4
 606 00c8 13F8143C 		ldrb	r3, [r3, #-20]	@ zero_extendqisi2
 607 00cc 4354     		strb	r3, [r0, r1]
 111:Src/StrBuf.c  ****             buf->array[(buf->ptr)++] = frac_digits[precision-1-i];
 608              		.loc 1 111 0 discriminator 4
 609 00ce 0132     		adds	r2, r2, #1
ARM GAS  /tmp/ccnzHx5Q.s 			page 14


 610              	.LVL62:
 611 00d0 D2B2     		uxtb	r2, r2
 612              	.LVL63:
 613              	.L36:
 111:Src/StrBuf.c  ****             buf->array[(buf->ptr)++] = frac_digits[precision-1-i];
 614              		.loc 1 111 0 is_stmt 0 discriminator 1
 615 00d2 1046     		mov	r0, r2
 616 00d4 3346     		mov	r3, r6
 617 00d6 F11B     		subs	r1, r6, r7
 618 00d8 8A42     		cmp	r2, r1
 619 00da 03DA     		bge	.L30
 111:Src/StrBuf.c  ****             buf->array[(buf->ptr)++] = frac_digits[precision-1-i];
 620              		.loc 1 111 0 discriminator 3
 621 00dc A988     		ldrh	r1, [r5, #4]
 622 00de EC88     		ldrh	r4, [r5, #6]
 623 00e0 A142     		cmp	r1, r4
 624 00e2 EAD3     		bcc	.L38
 625              	.LVL64:
 626              	.L30:
 627              	.LBE15:
 113:Src/StrBuf.c  ****     }
 114:Src/StrBuf.c  **** }
 628              		.loc 1 114 0 is_stmt 1
 629 00e4 07B0     		add	sp, sp, #28
 630              	.LCFI5:
 631              		.cfi_def_cfa_offset 36
 632              		@ sp needed
 633 00e6 BDE8F08F 		pop	{r4, r5, r6, r7, r8, r9, r10, fp, pc}
 634              	.LVL65:
 635              	.L47:
 636 00ea 00BF     		.align	2
 637              	.L46:
 638 00ec CDCCCCCC 		.word	-858993459
 639              		.cfi_endproc
 640              	.LFE8:
 642              		.section	.text.StrBuf_String,"ax",%progbits
 643              		.align	1
 644              		.global	StrBuf_String
 645              		.syntax unified
 646              		.thumb
 647              		.thumb_func
 648              		.fpu softvfp
 650              	StrBuf_String:
 651              	.LFB9:
 115:Src/StrBuf.c  **** 
 116:Src/StrBuf.c  **** void StrBuf_String(StrBuf *buf, const char *str)
 117:Src/StrBuf.c  **** {
 652              		.loc 1 117 0
 653              		.cfi_startproc
 654              		@ args = 0, pretend = 0, frame = 0
 655              		@ frame_needed = 0, uses_anonymous_args = 0
 656              		@ link register save eliminated.
 657              	.LVL66:
 658 0000 70B4     		push	{r4, r5, r6}
 659              	.LCFI6:
 660              		.cfi_def_cfa_offset 12
 661              		.cfi_offset 4, -12
ARM GAS  /tmp/ccnzHx5Q.s 			page 15


 662              		.cfi_offset 5, -8
 663              		.cfi_offset 6, -4
 664              	.LVL67:
 665              	.LBB16:
 118:Src/StrBuf.c  ****     for(uint32_t i = 0; str[i] && buf->ptr < buf->size; ++i)
 666              		.loc 1 118 0
 667 0002 0023     		movs	r3, #0
 668 0004 05E0     		b	.L49
 669              	.LVL68:
 670              	.L51:
 119:Src/StrBuf.c  ****         buf->array[(buf->ptr)++] = str[i];
 671              		.loc 1 119 0 discriminator 4
 672 0006 0568     		ldr	r5, [r0]
 673 0008 561C     		adds	r6, r2, #1
 674 000a 8680     		strh	r6, [r0, #4]	@ movhi
 675 000c 2478     		ldrb	r4, [r4]	@ zero_extendqisi2
 676 000e AC54     		strb	r4, [r5, r2]
 118:Src/StrBuf.c  ****     for(uint32_t i = 0; str[i] && buf->ptr < buf->size; ++i)
 677              		.loc 1 118 0 discriminator 4
 678 0010 0133     		adds	r3, r3, #1
 679              	.LVL69:
 680              	.L49:
 118:Src/StrBuf.c  ****     for(uint32_t i = 0; str[i] && buf->ptr < buf->size; ++i)
 681              		.loc 1 118 0 is_stmt 0 discriminator 1
 682 0012 CC18     		adds	r4, r1, r3
 683 0014 CA5C     		ldrb	r2, [r1, r3]	@ zero_extendqisi2
 684 0016 1AB1     		cbz	r2, .L48
 118:Src/StrBuf.c  ****     for(uint32_t i = 0; str[i] && buf->ptr < buf->size; ++i)
 685              		.loc 1 118 0 discriminator 3
 686 0018 8288     		ldrh	r2, [r0, #4]
 687 001a C588     		ldrh	r5, [r0, #6]
 688 001c AA42     		cmp	r2, r5
 689 001e F2D3     		bcc	.L51
 690              	.L48:
 691              	.LBE16:
 120:Src/StrBuf.c  **** }...
 692              		.loc 1 120 0 is_stmt 1
 693 0020 70BC     		pop	{r4, r5, r6}
 694              	.LCFI7:
 695              		.cfi_restore 6
 696              		.cfi_restore 5
 697              		.cfi_restore 4
 698              		.cfi_def_cfa_offset 0
 699 0022 7047     		bx	lr
 700              		.cfi_endproc
 701              	.LFE9:
 703              		.text
 704              	.Letext0:
 705              		.file 2 "/usr/include/newlib/machine/_default_types.h"
 706              		.file 3 "/usr/include/newlib/sys/_stdint.h"
 707              		.file 4 "Inc/StrBuf.h"
 708              		.file 5 "Inc/utils_mod.h"
ARM GAS  /tmp/ccnzHx5Q.s 			page 16


DEFINED SYMBOLS
                            *ABS*:0000000000000000 StrBuf.c
     /tmp/ccnzHx5Q.s:16     .text.StrBuf_Init:0000000000000000 $t
     /tmp/ccnzHx5Q.s:23     .text.StrBuf_Init:0000000000000000 StrBuf_Init
     /tmp/ccnzHx5Q.s:45     .text.StrBuf_Reset:0000000000000000 $t
     /tmp/ccnzHx5Q.s:52     .text.StrBuf_Reset:0000000000000000 StrBuf_Reset
     /tmp/ccnzHx5Q.s:69     .text.StrBuf_UsedSpace:0000000000000000 $t
     /tmp/ccnzHx5Q.s:76     .text.StrBuf_UsedSpace:0000000000000000 StrBuf_UsedSpace
     /tmp/ccnzHx5Q.s:92     .text.StrBuf_RemainingSpace:0000000000000000 $t
     /tmp/ccnzHx5Q.s:99     .text.StrBuf_RemainingSpace:0000000000000000 StrBuf_RemainingSpace
     /tmp/ccnzHx5Q.s:119    .text.StrBuf_Capacity:0000000000000000 $t
     /tmp/ccnzHx5Q.s:126    .text.StrBuf_Capacity:0000000000000000 StrBuf_Capacity
     /tmp/ccnzHx5Q.s:142    .text.StrBuf_Array:0000000000000000 $t
     /tmp/ccnzHx5Q.s:149    .text.StrBuf_Array:0000000000000000 StrBuf_Array
     /tmp/ccnzHx5Q.s:165    .text.StrBuf_UInt32:0000000000000000 $t
     /tmp/ccnzHx5Q.s:172    .text.StrBuf_UInt32:0000000000000000 StrBuf_UInt32
     /tmp/ccnzHx5Q.s:285    .text.StrBuf_UInt32:0000000000000078 $d
     /tmp/ccnzHx5Q.s:290    .text.StrBuf_UInt32Bin:0000000000000000 $t
     /tmp/ccnzHx5Q.s:297    .text.StrBuf_UInt32Bin:0000000000000000 StrBuf_UInt32Bin
     /tmp/ccnzHx5Q.s:434    .text.StrBuf_Float:0000000000000000 $t
     /tmp/ccnzHx5Q.s:441    .text.StrBuf_Float:0000000000000000 StrBuf_Float
     /tmp/ccnzHx5Q.s:638    .text.StrBuf_Float:00000000000000ec $d
     /tmp/ccnzHx5Q.s:643    .text.StrBuf_String:0000000000000000 $t
     /tmp/ccnzHx5Q.s:650    .text.StrBuf_String:0000000000000000 StrBuf_String

UNDEFINED SYMBOLS
cpow10
__aeabi_f2uiz
__aeabi_ui2f
__aeabi_fsub
__aeabi_fmul
